:020000020000FC
:100000000BC009C008C007C04AC105C004C003C076
:1000100002C001C000C018950BEF00936D0004E012
:10002000009362000093660003E0009369000EEF06
:100030000093600000E000936E0000936F00009357
:10004000700000937100009372000093730000939E
:1000500074000093640000936300009361000093B8
:100060006C0000936B0000936A000093680000939B
:100070006700009365000FED0DBF0FE907BB0FE7A9
:1000800001BB00E409BF0CE40BBD0BE40ABD78948E
:100090000EEF0093600010916100F0D006B3007283
:1000A0000030D9F400916F00003029F449D101E00B
:1000B00000936F0015C000916F00093649F00436B7
:1000C00019F40F933DD10F91039500936F0008C071
:1000D00037D105E600936F0003C000E000936F0086
:1000E00006B300740030D9F400917000003029F498
:1000F00053D101E00093700015C0009170000936E3
:1001000049F0043619F40F9347D10F9103950093EA
:10011000700008C041D105E60093700003C000E004
:1001200000937000F1D010916200A8D006B3007265
:100130000030D9F400917100003029F4ECD001E0D6
:100140000093710015C000917100093649F0043622
:1001500019F40F93E0D00F9103950093710008C03C
:10016000DAD005E60093710003C000E0009371004F
:1001700006B300740030D9F400917200003029F405
:10018000F4D001E00093720015C0009172000936AE
:1001900049F0043619F40F93E8D00F9103950093BA
:1001A000720008C0E2D005E60093720003C000E0D0
:1001B00000937200A9D01091630060D006B3007460
:1001C000003081F400917300003079F400916D00EB
:1001D0000270003011F44DD101C047D101E000930D
:1001E000730003C000E00093730006B30072003098
:1001F00019F500917400003011F500916E00003087
:1002000089F400E00DBD0CBD04E00EBD01E00093DB
:100210006E0000916D000270003011F4E5D001C055
:10022000D2D006C060D000E00EBD00E000936E00AA
:1002300001E00093740003C000E00093740064D0F8
:10024000109164001BD060D005D000916D0002BBFE
:100250005BD01ECF0FEF02BB0091600010916D00CC
:100260001470103021F410916E00103009F40F77E3
:1002700008BB000F01600093600008951F93EADF40
:100280001F91E4E9F2E020E0E10FF21FC895102D84
:1002900012BB0895C0F39492A38A88D3808200E0B1
:1002A0000CBD0DBD00916D0001700030D1F00091CA
:1002B0006400003079F400916300003059F400913B
:1002C0006200003031F400916100003011F411D06F
:1002D00002C062D04AD000916D000E7F00936D0085
:1002E00001C001D0189500916D00016000936D0070
:1002F000089500916D000270003019F486D0AED0E0
:1003000002C094D0A4D0089510E028E21A95F1F725
:100310002A95E1F708950091640003950093640025
:100320000A3069F400E000936400009163000395D3
:1003300000936300063019F400E000936300089511
:10034000009162000395009362000A3069F400E0B6
:1003500000936200009161000395009361000A30F0
:1003600019F400E0009361000895009164000030EA
:1003700021F00A95009364000EC009E00093640028
:1003800000916300003021F00A950093630003C0E0
:1003900005E000936300089500916200003021F0B1
:1003A0000A95009362000EC009E00093620000917C
:1003B0006100003021F00A950093610003C009E05C
:1003C0000093610008950091610000936500009121
:1003D0006200009366000091630000936700009143
:1003E0006400009368000895009161000093690023
:1003F0000091620000936A000091630000936B001B
:100400000091640000936C000895009165000093D2
:100410006100009166000093620000916700009304
:1004200063000091680000936400089500916900E2
:100430000093610000916A000093620000916B00DC
:100440000093630000916C00009364000895009194
:100450006D0004600D7F00936D00089500916D00A4
:1004600002600B7F00936D000895ADDFDFDFEFDFEB
:0A0470000895BADFCADFF2DF089535
:00000001FF
